:020000000F28C7
:10000800DE00030E8312A1000408A2000A08A30060
:100018005F08A40062288316FF2390008312142827
:10002800AA01A601A701A80183011A288B0107309C
:1000380083129900013085000130831685008430D1
:1000480081007D308312A5002508A900A7012A1088
:10005800A801A601063081008B168B172A1C3728A9
:1000680083128514392883128510051858287D3085
:10007800A5002508A800A60105184528A808031DFD
:100088004028A80803195828051C4D28A808031D4E
:100098004828A808031958280130A5002508A607EC
:1000A80005302602031C402805302602031C602860
:1000B800A6010130AA063228A60132280B1D812884
:1000C8000B11063081000130A902280803196E2897
:1000D8000130A802A908031D79287D30A000200856
:1000E800A9000430A0002008A700270803198028C9
:1000F8000130A7020515812805112408DF0023080F
:100108008A0022088400210E8300DE0E5E0E09009C
:02400E00E1319E
:00000001FF
